:020000040000FA
:100000008316031318280000B2000308B3008316F8
:1000100003131530811D03018312031381000B119B
:10002000B008031DB00333088300B20E320E09007E
:100030000E309F005730810021308500FF30860050
:1000400080308700243098000A309900831203130F
:1000500080309F0090309800FF3085008600870038
:10006000203084008001840A34300402031D3228C9
:100070000B308700A50005120000051600001030A7
:100080008700A40005120000051600002330870039
:10009000A300051200000516000030308700A20002
:1000A000051200000516000003018100A0308B003E
:1000B0001A08B008031D6C281730B0000511851010
:1000C00000000000060805158514B1002E02031972
:1000D0006C283108AE00A2228C1E592818197E28DF
:1000E00098187E288B131A08A00082208316031309
:1000F00057308100831203138B1759281A081812DE
:100100001816592800308A0020080F398207A428C1
:10011000AC28B428BC28C428C628D529D729762AD3
:10012000CA28CE280800080008000800080000308F
:100130008A002408073982070134023404340A345F
:10014000143428346434C834200E8700A500051206
:100150000000051600000729200E8700A4000512E4
:100160000000051600000729200E8700A3000512D5
:100170000000051600000729200E8700A2000512C6
:1001800000000516000007298622C7288E22211CA0
:10019000D1280A29200E0139A10007299622AF0093
:1001A000072903308700A50005120000051600008E
:1001B0000511851405308700A500051200000516FD
:1001C00000008C1EF8281819F5289818F5281A0828
:1001D0000E3C031DF8280B308700A5000512000017
:1001E000051600001530A22208001A081812181669
:1001F000851EE1280000851EE1280000851EE128FB
:100200000B308700A500051200000516000006301F
:10021000A22208000515851081309F00A1132F0828
:10022000AD002808A6002908A700A60F1829A70ACC
:10023000831603135F308100831203139C30810007
:100240000B11013024299720B0008B17B008031D33
:1002500026298B1300007B21A11F4B298316031332
:100260008601831203132B08860000008511851573
:100270002D08860000008511851583160313860955
:1002800083120313A60B4829A708031D4B297829BD
:1002900026090319A7038C1E702918196D299818AF
:1002A0006D291A080E3C031D70290B308700A5002C
:1002B000051200000516000080309F000230A222C7
:1002C0002608A802031CA9032708A9022908A222BC
:1002D0002808A2220330A22208001A0818121816B1
:1002E000851E23290000851E23290000851E232941
:1002F00080309F0000291F152D08AC002B08AA0094
:1003000001308700A500051200000516000000005E
:100310000608AB0009308700A5000512000005168D
:1003200000001F1991291E08AD00A11B0800A41D83
:100330009B29A117080023080339031DA4292D08B0
:100340002F020318A1170800B100B10BB0292C0827
:100350002F02031808002D082F020318BF290800D8
:10036000B10BB7292F082D020318A11708002F0879
:100370002C02031808002F082D02031C0800A117E7
:10038000831603138601831203132A0886000000D4
:10039000851185152C0886000000851185158316AA
:1003A000031386098312031308008622D8298E229C
:1003B0000B308700A5000512000005160000211C67
:1003C000E42905158510E629051185140230A222BD
:1003D0002708A2222608A22208308700A5000512BD
:1003E000000005160000000000000608AA00A22276
:1003F00009308700A5000512000005160000211C29
:10040000552A0000000008308700A50005120000F2
:1004100005160000000000000608AC00A22209300A
:100420008700A5000512000005160000552A0830B7
:100430008700A5000512000005160000000000005E
:100440000608AB0009308700A5000512000005165C
:100450000000211C3F2A0000000008308700A50092
:100460000512000005160000000000000608AD009F
:1004700009308700A50005120000051600002B08B2
:100480002A02031D492A211C552A2D082C02031972
:10049000552A2708A2222608A2222B08AA00A22257
:1004A000211C552A2D08AC00A222A60F582AA70A03
:1004B00027082902031C622A031D172A260828027E
:1004C0000318172A2908A2222808A2222B08A222F0
:1004D000211C6C2A2D08A2220B308700A5000512D2
:1004E0000000051600008030A22208000230A2227F
:1004F000240EA222230EA222220EA222210E0938AD
:10050000A2222F08A2220330A22208000030A60057
:10051000A700FF30A8007F30A90008009622A9009C
:100520009622A8000030A600A70008008C1E962A7C
:1005300018199E2A98189E2A1A0808001A081812D4
:100540001816962A83160313981CA42A83120313E1
:040550009900080006
:02400E00323F3F
:00000001FF
